:100000000C9442010C946A010C946A010C946A01EC
:100010000C946A010C946A010C946A010C946A01B4
:100020000C946A010C946A010C94290A0C949B0AA2
:100030000C946A010C946A010C946A010C946A0194
:100040000C946A010C946A010C946A010C946A0184
:100050000C946A010C946A010C946A010C94760E5B
:100060000C946A010C946A010C946A010C946A0164
:100070000C946A010C946A010C946A010C946A0154
:100080000C946A010C946A010C946A010C946A0144
:100090000C946A010C946A010C946A010C946A0134
:1000A0000C946A010C946A010C946A01414C41520F
:1000B0004D00414C4C004D4944444C450052494789
:1000C0004854004C45465400414C4C004D49444472
:1000D0004C45005249474854004C45465400414C59
:1000E0004C004D4944444C45005249474854004C4B
:1000F0004546540000000000000000002A2B2800A4
:1001000000000000000000000000000000000000EF
:10011000000000002C9EB4A0A1A2A434A6A7A5AE06
:10012000362D3738271E1F20212223242526B333BE
:10013000B62EB7B89F8485868788898A8B8C8D8EEA
:100140008F909192939495969798999A9B9C9D2FB6
:100150003130A3AD350405060708090A0B0C0D0E56
:100160000F101112131415161718191A1B1C1DAF96
:10017000B1B0B500080B0002020201000904000042
:100180000102020000052400100105240101010400
:10019000240206052406000107058103100040091A
:1001A000040100020A0000000705020240000007E7
:1001B0000583024000000403090412010002EF025B
:1001C0000140412336800001010203014172647540
:1001D000696E6F204C4C430041726475696E6F20EC
:1001E0004C656F6E6172646F00636C69636B007263
:1001F000656C65617365007072657373006D6F7611
:1002000065006B7772697465006B72656C6561730C
:1002100065006B70726573730053455400050109E6
:1002200002A1010901A10085010509190129031590
:10023000002501950375018102950175058103056E
:10024000010930093109381581257F750895038129
:1002500006C0C005010906A1018502050719E029AC
:10026000E715002501750195088102950175088142
:100270000395067508150025730507190029738174
:1002800000C0641111241FBECFEFDAE0DEBFCDBF86
:1002900023E0AEE8B2E001C01D92A736B207E1F755
:1002A00012E0A0E0B1E0E8EAF9E202C005900D92A8
:1002B000AE38B107D9F711E0C2E4D1E004C021970C
:1002C000FE010E94D012C134D107C9F70E94C00EAE
:1002D0000C94D2140C9400004091B5025091B602D7
:1002E0002091B3023091B40242175307B4F49091B5
:1002F000E8009570E1F39091E80092FD19C08093B9
:10030000F1008091B5029091B60201968F73992702
:10031000892B19F48EEF8093E8008091B5029091BB
:10032000B60201969093B6028093B50281E00895DB
:1003300080E008952FB7F89487708093E90090913A
:10034000E800892F807295FF04C09091F20080E44C
:10035000891B2FBF0895CF92DF92EF92FF920F93E8
:100360001F93CF93DF936C017A018B01C0E0D0E043
:10037000CE15DF0581F0D8016D918D01D601ED918B
:10038000FC910190F081E02DC6010995892B11F0B7
:100390002196EECF7E01C701DF91CF911F910F9182
:1003A000FF90EF90DF90CF900895CF93DF931F924F
:1003B000CDB7DEB76983DC01ED91FC910280F3815A
:1003C000E02D41E050E0BE016F5F7F4F09950F9037
:1003D000DF91CF91089583E08093E9008091F2004E
:1003E000882319F08AE38093E800089583E00E944F
:1003F0009A0190E00895FC018485958597FD0BC0D6
:100400009FB7F89482E08093E9008091F2009FBF4B
:1004100090E0019608959FB7F89482E08093E900F8
:100420008091F2009FBF90E00895DC01FB011296DD
:100430008C91129790E02481358182179307D1F433
:1004400091818081813A31F481E0913091F0933053
:1004500089F411C0813271F49B3021F482811F969E
:100460008C9305C09A3031F4828150968C9381E050
:100470000895089580E00895DC01FB0188E48083FD
:1004800089E4818384E482831D969C911D979F70EB
:100490009F5B93831D968D919C911E9724E096956A
:1004A00087952A95E1F78F708F5B848385E00895A7
:1004B000FC0182818F5BFB01808381E00895CF92F4
:1004C000DF92EF92FF920F931F93CF93DF936C0114
:1004D000EB017B01E40EF51E00E010E0CE15DF0518
:1004E00081F069916D30D1F3D601ED91FC910190CD
:1004F000F081E02DC6010995892B19F00F5F1F4F80
:10050000EDCFC801DF91CF911F910F91FF90EF9038
:10051000DF90CF900895089580E090E00895EF92E5
:10052000FF920F931F93CF93DF938C017B01C0E069
:10053000D0E0D801ED91FC910680F781E02DBE015D
:10054000C8010995882371F0D801ED91FC910084D0
:10055000F185E02DA701BE01C8010995811102C0F6
:100560002196E7CFDF91CF911F910F91FF90EF90F0
:1005700008956830710580F4675F7F4F660F771FBD
:10058000FC01E60FF71F0190F081E02D309721F07C
:10059000CA01099581E0089580E0089568307105E9
:1005A00060F46F5F7F4F660F771FFC01E60FF71F48
:1005B00081E020813181232B09F480E0089588E0D7
:1005C00090E0089580E490E00895079608950F93D1
:1005D0001F93CF93DF931F92CDB7DEB78C01FC0141
:1005E0008485958597FF0EC0CE0101960E94480E26
:1005F000019719F4898190E002C08FEF9FEFF80115
:1006000095878487F801848595850F90DF91CF9138
:100610001F910F910895CF93DF931F92CDB7DEB74F
:10062000FC018485958597FD05C02FEF3FEF358749
:1006300024870BC0CE0101960E94480E019719F441
:10064000898190E002C08FEF9FEF0F90DF91CF91F3
:100650000895EF92FF920F931F93CF93DF937C0146
:10066000EB018A01DC01ED91FC910680F781E02D20
:100670000995282F882371F02196CC0FDD1FCE0D10
:10068000DF1D68817981C8010E943C1221E0892B1D
:1006900009F020E0822FDF91CF911F910F91FF9001
:1006A000EF900895079621E4FC0111922A95E9F74D
:1006B0000895DF92EF92FF920F931F93CF93DF93F2
:1006C000D82EF92EE42E062F10E0C8010196880FCF
:1006D0000E946C0183E00E946C01CD2DDF2D0C0F78
:1006E0001D1FC017D10789F0E7FE03C0FE018491EA
:1006F00001C088810E946C01F82E80E00E946C018C
:100700008F2121968111EDCF01C081E0DF91CF9142
:100710001F910F91FF90EF90DF900895DF92EF927D
:10072000FF920F931F93CF93DF93D82E8A017B0103
:10073000E40EF51EEB01CE15DF0571F0D7FE03C008
:10074000FE01849101C088810E946C012196811173
:10075000F2CF8FEF9FEF01C0C801DF91CF911F91C2
:100760000F91FF90EF90DF900895EF92FF920F931B
:100770001F93CF93DF93FB012081213851F5238113
:10078000223239F5DC0112962C9130E044815581FA
:1007900042175307F1F4EC010B851C85E12CF12C79
:1007A0000115110591F0F801448155816281738131
:1007B00080E80E948E038F3FFFEF9F0769F0E80EED
:1007C000F91ED8010D911C91EBCF81E08F87C701F5
:1007D00005C080E090E002C08FEF9FEFDF91CF91E6
:1007E0001F910F91FF90EF900895CF93DF93CDB7B6
:1007F000DEB769970FB6F894DEBF0FBECDBFFC0120
:10080000DB018C918F5F8C93BE016F5F7F4F89E11D
:10081000DB011D928A95E9F729E0298384E08A8328
:1008200091E09D8383E08E832A8721E22B879C873A
:100830009D879F8722E2288B27E02B8B25E02C8B3E
:100840008E8B20E430E0388F2F8B998F82818B83C1
:1008500095858685998B8A8B838180688D8B49E10C
:1008600050E080E00E948E0369960FB6F894DEBFD8
:100870000FBECDBFDF91CF9108957F928F929F924F
:10088000AF92BF92CF92DF92EF92FF920F931F939E
:10089000CF93DF93C82E8B017A018091BC02811126
:1008A00003C08FEF9FEF70C08091B80280FF05C03A
:1008B0008091E00082608093E000CE2DDF2DD12C6E
:1008C0008AEFB82E8C2D8770982E8C2D8072882EF2
:1008D0008C2D8074782E9AE3A92E209719F4DD20B0
:1008E00009F44DC08C2D0E949A01811106C0BA9462
:1008F000BB20B9F20E947B0DF0CF282F30E0C21749
:10090000D3070CF48C2F9FB7F8949092E9002091B4
:10091000E80025FF32C0282F30E0C21BD30B88200F
:1009200029F08150A0F01092F100FBCFF801C7FE32
:100930000AC0815050F044914093F1003196F9CFB4
:1009400041914093F1008150D8F7020F131FDD2031
:1009500019F0A092E8000AC08091E80085FD08C067
:10096000A092E800DD24D394209739F0D12C05C063
:10097000209719F47110A092E8009FBFAECF5D9848
:1009800084E68093B702C701DF91CF911F910F9149
:10099000FF90EF90DF90CF90BF90AF909F908F909F
:1009A0007F900895CF93DF93EC018091120188230B
:1009B00031F083E00E943D041816190634F081E0FE
:1009C00090E09B838A8380E090E0DF91CF9108954F
:1009D000615030F02091F100FC0120830196F8CFA6
:1009E000289884E68093BB0208958091AB02811120
:1009F0000DC082E08093A70284E08093A802109249
:100A0000AA021092A90281E08093AB0287EA92E0E9
:100A1000089580919F0281116AC081E080939202C3
:100A20008093930228E932E0309395022093940258
:100A300010929702109296022DE131E030938F02CE
:100A400020938E0210929A021092990210929C02A8
:100A500010929B0280939D0280939E0281EC809372
:100A600098020E94F504FC0121818091920290E09D
:100A7000820F911D0897C4F5A281B381109729F4C4
:100A80008EE892E0938382830EC018968D919C919C
:100A90001997009711F0DC01F8CF8EE892E01996D3
:100AA0009C938E931897808180939002818180938C
:100AB0009102908180919302890F808380E09091D0
:100AC0009202891788F4A0919402B0919502A80F20
:100AD000B11D9C91A181B0E0A050BF4F9C9391812A
:100AE0009F5F91838F5FEBCF81E080939F028EE8C1
:100AF00092E00895CF93DF93DC01683810F06858D6
:100B00002DC0E62FF0E067FF11C0E058F10981E049
:100B100090E001C0880FEA95EAF714969C9114972B
:100B2000892B14968C93149760E018C0EC50FF4FFB
:100B30006491611109C081E090E013969C938E93BB
:100B4000129780E090E046C067FF08C014968C9131
:100B50001497826014968C9314976F7716968C91E5
:100B60001697681751F117968C911797681729F106
:100B700018968C911897681701F119968C9119970E
:100B80006817D9F01A968C911A976817B1F01B96CE
:100B90008C911B97681789F0FD01369680E090E0F4
:100BA0002191211105C0FD01E80FF91F668305C0E1
:100BB000019686309105A1F7BECFED010E9409058F
:100BC000AE014C5F5F4F28E030E062E00E94950D7F
:100BD00081E090E0DF91CF910895CF93DF93DC0126
:100BE000683810F0685825C0E62FF0E067FF12C0A3
:100BF000E058F10981E090E001C0880FEA95EAF73A
:100C0000809514969C911497892314968C9314972D
:100C100060E00FC0EC50FF4F6491662321F167FF45
:100C200008C014968C9114978D7F14968C9314970A
:100C30006F77FD0186E0662321F09681691301C07C
:100C40001682815031968111F6CFED010E9409057F
:100C5000AE014C5F5F4F28E030E062E00E94950DEE
:100C600081E090E002C080E090E0DF91CF910895B4
:100C7000EF92FF921F93CF93DF93EC01162F0E9408
:100C80007A057C01612FCE010E94ED05C7019927ED
:100C9000DF91CF911F91FF90EF900895CF93DC01EA
:100CA00017968D919C9118978617970758F115966E
:100CB0008D919C91169720E030E040E050E028179D
:100CC000390701F12115310581F01396ED91FC9161
:100CD0001497E20FF31FC081C11117C03197E08153
:100CE000EE2369F04F5F5F4F0AC04617570739F48C
:100CF0001396ED91FC911497C081C11109C02F5F2B
:100D00003F4FDDCFE0E0F0E003C046175707B9F7EB
:100D1000CF01CF910895CF92DF92EF92FF920F9380
:100D20001F93CF93DF93EC016B0160E070E0C6018D
:100D30000E944E067C01892B59F100E010E0E88109
:100D4000F9810680F781E02DB801CE01099588234D
:100D5000F9F0E881F9810084F185E02DA701B8015F
:100D6000CE010995882389F0E881F9810284F38511
:100D7000E02DA601B801CE01DF91CF911F910F9117
:100D8000FF90EF90DF90CF9009940F5F1F4FD7CF68
:100D900080E0DF91CF911F910F91FF90EF90DF9056
:100DA000CF9008950F931F93CF93DF93CDB7DEB706
:100DB0002C970FB6F894DEBF0FBECDBF8C0161E05B
:100DC00070E00E944E06BC01CE0101960E94EE0921
:100DD000CE0101960E94E60D8EE093E00E94380657
:100DE000CE0101960E94060D61E070E0C8010E94EC
:100DF0004E06BC01CE0107960E94EE096DE571E03A
:100E0000CE0101960E94EE09BE01695F7F4FCE01BF
:100E100001960E941E0D0E940B0DCE0101960E94AC
:100E2000060DCE0107960E94060D2C960FB6F8947B
:100E3000DEBF0FBECDBFDF91CF911F910F910895FF
:100E40000F931F93CF93DF93CDB7DEB72C970FB6D9
:100E5000F894DEBF0FBECDBF8C0161E070E00E9450
:100E60004E06BC01CE0101960E94EE09CE0101960C
:100E70000E94E60D8EE093E00E94ED05CE01019602
:100E80000E94060D61E070E0C8010E944E06BC01A0
:100E9000CE0107960E94EE0964E671E0CE0101964C
:100EA0000E94EE09BE01695F7F4FCE0101960E944C
:100EB0001E0D0E940B0DCE0101960E94060DCE0163
:100EC00007960E94060D2C960FB6F894DEBF0FBE53
:100ED000CDBFDF91CF911F910F9108950F931F9375
:100EE000CF93DF93CDB7DEB72C970FB6F894DEBF64
:100EF0000FBECDBF8C0161E070E00E944E06BC01C8
:100F0000CE0101960E94EE09CE0101960E94E60DE7
:100F10008EE093E00E947A05CE0101960E94060DB4
:100F200061E070E0C8010E944E06BC01CE01079648
:100F30000E94EE096DE671E0CE0101960E94EE0975
:100F4000BE01695F7F4FCE0101960E941E0D0E9477
:100F50000B0DCE0101960E94060DCE0107960E9450
:100F6000060D2C960FB6F894DEBF0FBECDBFDF91F5
:100F7000CF911F910F910895CF93DF93EC016FEE06
:100F800070E00E940D0E882331F081E00E943A0E3D
:100F900084E791E02CC069EE70E0CE010E940D0E56
:100FA000882331F082E00E943A0E85E891E01FC06C
:100FB00062EE70E0CE010E940D0E882331F084E0D5
:100FC0000E943A0E87E991E012C06EED70E0CE010A
:100FD0000E940D0E882331F087E00E943A0E8AEAC3
:100FE00091E005C061E070E0CE010E944E06DF9105
:100FF000CF910C94F10DCF93DF93EC0169ED70E08C
:101000000E940D0E882331F081E00E942C0E8AEBA5
:1010100091E02CC063ED70E0CE010E940D0E88239C
:1010200031F082E00E942C0E8DEC91E01FC06CEC40
:1010300070E0CE010E940D0E882331F084E00E9402
:101040002C0E81EE91E012C068EC70E0CE010E949F
:101050000D0E882331F087E00E942C0E86EF91E080
:1010600005C061E070E0CE010E944E06DF91CF9195
:101070000C94F10DCF93DF93EC0163EC70E00E94D0
:101080000D0E882331F081E00E941F0E88E092E06F
:101090002CC06DEB70E0CE010E940D0E882331F064
:1010A00082E00E941F0E89E192E01FC066EB70E0B3
:1010B000CE010E940D0E882331F084E00E941F0EA5
:1010C0008BE292E012C062EB70E0CE010E940D0E46
:1010D000882331F087E00E941F0E8EE392E005C066
:1010E00061E070E0CE010E944E06DF91CF910C943A
:1010F000F10DCF92DF92EF92FF920F931F93CF9358
:10110000DF93CDB7DEB768970FB6F894DEBF0FBE9A
:10111000CDBF8C0161E070E00E944E06BC01CE01A3
:1011200001960E94EE09CE0101960E94E60DF62E70
:10113000D72ECE0101960E94060D62E070E0C80134
:101140000E944E06BC01CE0101960E94EE09CE011E
:1011500001960E94E60DE62EC72ECE0101960E9452
:10116000060D63E070E0C8010E944E06BC01CE018E
:1011700001960E94EE09CE0101960E94E60D162FFF
:10118000072FCE0101960E94060D412F6E2D8F2D47
:101190000E94C90D612F702FCE0143960E94310D20
:1011A0006E2D7C2DCE010D960E94310D6F2D7D2D63
:1011B000CE0107960E94310D6EE472E0CE010196D9
:1011C0000E94EE09BE01695F7F4FCE0101960E9429
:1011D0001E0D64E572E00E94D509BE01635F7F4F7A
:1011E0000E941E0D64E572E00E94D509BE016D5E8D
:1011F0007F4F0E941E0D67E572E00E94D5090E9494
:101200000B0DCE0101960E94060DCE0107960E949D
:10121000060DCE010D960E94060DCE0143960E944A
:10122000060D68960FB6F894DEBF0FBECDBFDF91F6
:10123000CF911F910F91FF90EF90DF90CF90089585
:10124000CF93DF93EC0189E592E00E94F10D6CEA07
:1012500070E0CE010E940D0E882331F062E070E054
:10126000CE010E944E0602C085E692E0DF91CF914A
:101270000C94F10D0E94BD140F931F93CF93DF9335
:101280001F92CDB7DEB782E0898342E450E064E785
:1012900071E080E80E948E030E94F504DC01129642
:1012A0000D911C9113970115110589F0D801ED914D
:1012B000FC910280F381E02DBE016F5F7F4FC8017A
:1012C000099597FD04C0F80100851185ECCF89814F
:1012D0000F90DF91CF911F910F9108950F931F935E
:1012E000CF93DF93EC0188819981009729F02A81BF
:1012F0003B812617370788F48B016F5F7F4F0E9471
:10130000F713009761F0998388831B830A832C81EC
:101310003D81232B11F4FC01108281E001C080E0AB
:10132000DF91CF911F910F910895EF92FF920F934C
:101330001F93CF93DF936115710511F480E01CC0FA
:1013400041155105C1F07B01EC018C819D818A0121
:10135000080F191FB801CE010E946E09882371F38E
:10136000288139818C819D81B701820F931F0E9452
:10137000CB141D830C8381E0DF91CF911F910F91DE
:10138000FF90EF900895CF93DF93EC0188819981CE
:10139000009711F00E946E13198218821D821C8220
:1013A0001B821A82DF91CF910895CF93DF93EC01D6
:1013B0006115710561F0FB0101900020E9F731979B
:1013C000AF01461B570B0E949509811103C0CE0146
:1013D0000E94C309CE01DF91CF910895EF92FF9251
:1013E0000F931F93CF93DF93EC01198218821B8216
:1013F0001A821D821C826115710521F18B01FB018E
:1014000001900020E9F731977F01E61AF70AB7014A
:101410000E946E09811109C0CE01DF91CF911F9109
:101420000F91FF90EF900C94C309FD82EC82B801FC
:1014300088819981DF91CF911F910F91FF90EF905B
:101440000C94CB14DF91CF911F910F91FF90EF90EF
:1014500008951F920F920FB60F9211248F939F93AE
:101460008091E1009091E100937F9093E10083FFF0
:101470000FC01092E90091E09093EB001092EC0005
:1014800092E39093ED001092BC0298E09093F000EC
:1014900082FF20C093E09093E9009091F20099239D
:1014A00019F09AE39093E8009091B702992339F0EC
:1014B0009091B70291509093B702992389F190913E
:1014C000BB02992339F09091BB0291509093BB02DB
:1014D000992341F184FF10C08091E2008E7E8160EB
:1014E0008093E2008091E1008F7E8093E100809103
:1014F000B8028E7E806111C080FF16C08091E2002C
:101500008E7E80618093E2008091E1008E7E8093E8
:10151000E1008091B8028E7E81608093B80204C0A1
:101520005D9ACDCF289AD6CF9F918F910F900FBE05
:101530000F901F9018951F920F920FB60F921124C3
:10154000CF92DF92EF92FF920F931F932F933F93CF
:101550004F935F936F937F938F939F93AF93BF93BB
:10156000EF93FF93CF93DF93CDB7DEB76C97DEBFDA
:10157000CDBF1092E9008091E80083FFFBC168E0D5
:10158000CE0145960E94E80482EF8093E8008D89A1
:1015900087FF05C09091E80090FFFCCF03C09EEF4D
:1015A0009093E800982F907609F0C6C09E894F89E5
:1015B000588D2F89F88C91110CC0803829F48091B6
:1015C000BA028093F10002C01092F1001092F10073
:1015D00045C1913051F4811141C14130510509F0AB
:1015E0003DC18091BA028D7F0BC0933061F48111AF
:1015F00035C14130510509F031C18091BA02826094
:101600008093BA022BC1953049F48091E80080FFA5
:10161000FCCF822F80688093E30020C1963009F0D0
:101620005EC00B8D1C8D22E01092E9001092B60274
:101630001092B502F21232C01092B4021092B302AC
:101640000E943C0999E0BE016F5F7F4FDB01E92FEB
:101650001D92EA95E9F79983FA8291E09E8390EAD8
:1016600098879AEF99872091B5023091B602275F4B
:101670003F4F3C832B838D831092E9001092B6027A
:101680001092B5021093B4020093B30249E050E007
:1016900080E00E948E030E943C09E0C01093B402D7
:1016A0000093B3020E94F504DC0112960D911C9187
:1016B00013970115110509F4BBC0D801ED91FC91F8
:1016C0000480F581E02DBE016B5E7F4FC801099556
:1016D000009709F0C7C0F80100851185EACF97305F
:1016E00009F445C1983021F481E08093F100B6C03F
:1016F000993009F0B3C0837009F039C1E1E0F1E03D
:1017000081E031E096E32081211109C08EE78093CA
:10171000EA001092EA008F898093BC029FC08093F8
:10172000E9003093EB0021912093EC009093ED00C1
:101730008F5F873041F7EACF8B8D9C8D1092E90047
:101740001092B6021092B5029093B4028093B30245
:10175000898D811153C08E899D89913A49F48132D6
:1017600009F005C147E050E06BE071E080E0BBC0EC
:10177000913209F0FCC0833269F48F89988DA0E022
:10178000B0E08093070190930801A0930901B09302
:101790000A0164C0803269F48091E80082FFFCCFC6
:1017A00067E08BE091E00E94E8048BEF8093E80013
:1017B00055C0823209F052C08F8980931201EEEF3A
:1017C000FFE7859194918B3F9C4D19F0E0E0F8E0A4
:1017D00002C0EEEFFAE080910B0190910C01A09114
:1017E0000D01B0910E01803B9440A105B10509F0B7
:1017F0009EC08091120180FF79C099C00E94F504BB
:10180000FC01028113810115110509F4B0C0D80152
:10181000ED91FC910190F081E02DBE016B5E7F4F58
:10182000C801099581111AC0F80100851185EBCF17
:10183000F1E0FF1609F44EC0F3E0FF1298C08F8963
:10184000882309F44AC0823089F440E860E188EDD9
:1018500091E00E945903882309F489C08EEF809398
:10186000E80088C018161906CCF381C0813029F42D
:1018700040E86BE08CEC91E0ECCF833009F077C06E
:101880000E94F504DC011296ED90FC9013978E01F6
:101890000F5F1F4F6801E114F10479F0D701ED915A
:1018A000FC910680F781E02DB801C7010995080F6A
:1018B000111DF701E084F184EECFD8011C92F601EE
:1018C00001900020E9F73197BF016C197D0940E0D4
:1018D000C601BFCF6AEB71E002C066EB71E0FB01AD
:1018E000449150E080E80E948E03B8CFEE3F2AE09A
:1018F000F20751F0808191818737A7E79A0721F09D
:101900009093FF0A8093FE0A87E797E7918380838D
:10191000809160008093B9029BE088E10FB6F89453
:10192000A895809360000FBE9093600097CF808150
:1019300091818737974709F091CFA89580916000F2
:101940008861809360008091B90280936000EE3FCF
:10195000BAE0FB0739F08091FE0A9091FF0A91836B
:1019600080837CCF1092FF0A1092FE0A77CF81E22B
:101970008093EB006C960FB6F894DEBF0FBECDBF20
:10198000DF91CF91FF91EF91BF91AF919F918F9197
:101990007F916F915F914F913F912F911F910F9187
:1019A000FF90EF90DF90CF900F900FBE0F901F90A1
:1019B00018953FB7F8948091430390914403A09108
:1019C0004503B091460326B5A89B05C02F3F19F0EB
:1019D0000196A11DB11D3FBFBA2FA92F982F8827AF
:1019E000820F911DA11DB11DBC01CD0142E0660F0A
:1019F000771F881F991F4A95D1F7089542E050E05C
:101A00006AE872E08DEB92E00C94D204FC018081D4
:101A100091810C946E13CF93DF93FC014481558127
:101A2000608171818DEB92E00E94D204EC010E94F2
:101A3000FE0C8C0F9D1FDF91CF910895CF93DF9304
:101A4000EC01FB0144815581608171810E949509FF
:101A5000811103C0CE010E94C309CE01DF91CF9155
:101A60000895CF92DF92EF92FF920F931F93CF933F
:101A7000DF93CDB7DEB762970FB6F894DEBF0FBE27
:101A8000CDBF8C01CB01F80111821082138212822A
:101A9000158214824AE09E012F5F3F4F6901B90110
:101AA0000E944F12F60101900020E9F731977F0163
:101AB000EC18FD08B701C8010E946E09811104C02D
:101AC000C8010E94C30908C0F801F582E482B6018A
:101AD000808191810E94CB1462960FB6F894DEBF8C
:101AE0000FBECDBFDF91CF911F910F91FF90EF906F
:101AF000DF90CF900895CF92DF92EF92FF920E94F5
:101B0000D90C6B017C010E94D90CDC01CB018C1932
:101B10009D09AE09BF09883E9340A105B10598F320
:101B2000FF90EF90DF90CF900895AF92BF92CF9249
:101B3000DF92EF92FF920F931F93CF93DF931F9249
:101B4000CDB7DEB77C0169836A01590141E050E0FD
:101B5000BE016F5F7F4FFC0183810E943D048C01B9
:101B600097FD0BC0F7018381A501B60180640E9437
:101B70003D0497FD02C0800F911F0F90DF91CF9120
:101B80001F910F91FF90EF90DF90CF90BF90AF909B
:101B90000895CF93DF9300D000D0CDB7DEB79091FA
:101BA0000D0399838A836B834C830E94090524E08B
:101BB00030E0AE014F5F5F4F61E00E94950D0F90E6
:101BC0000F900F900F90DF91CF910895FC018081CD
:101BD0009181009711F00C94151260E070E0CB0138
:101BE0000895CF93DF93009779F0FC0101900020D6
:101BF000E9F73197AF01481B590BBC018DEB92E01F
:101C00000E94D204EC0102C0C0E0D0E00E94FE0CB1
:101C10008C0F9D1FDF91CF910895CF93DF93EB0140
:101C200061E070E00E944E06BE010E943C1221E07D
:101C3000892B09F020E0822FDF91CF9108959091B8
:101C40000D03892B981739F080930D0340E060E075
:101C500080E00C94C90D089590910D03809589231F
:101C6000981739F080930D0340E060E080E00C9419
:101C7000C90D089580930D0340E060E080E00E946C
:101C8000C90D10920D0340E060E080E00C94C90D96
:101C90002091BC02211103C08FEF9FEF08955FB721
:101CA000F89422E02093E9002091F20030E012162F
:101CB000130614F421E030E0422FFC0184E6415089
:101CC00038F028988093BB029091F1009193F7CF60
:101CD0002115310521F08091F200882319F05FBFB2
:101CE000C90108958BE68093E800F9CF1F920F9207
:101CF0000FB60F9211242F933F938F939F93AF931F
:101D0000BF9380913F0390914003A0914103B09114
:101D1000420330913E0323E0230F2D3720F4019638
:101D2000A11DB11D05C026E8230F0296A11DB11DFE
:101D300020933E0380933F0390934003A09341037D
:101D4000B09342038091430390914403A0914503D3
:101D5000B09146030196A11DB11D8093430390935A
:101D60004403A0934503B0934603BF91AF919F9165
:101D70008F913F912F910F900FBE0F901F9018954C
:101D8000CF93DF93CDB7DEB7C155D1090FB6F89425
:101D9000DEBF0FBECDBF789484B5826084BD84B5AC
:101DA000816084BD85B5826085BD85B5816085BD56
:101DB00080916E00816080936E001092810080910E
:101DC0008100826080938100809181008160809396
:101DD00081008091800081608093800080919100DB
:101DE0008260809391008091910081608093910046
:101DF000809190008160809390008091C100846008
:101E00008093C1008091C10082608093C100809165
:101E1000C10081608093C1008091C3008160809384
:101E2000C3008091C00082608093C0008091C20096
:101E300081608093C20080917A00846080937A00F0
:101E400080917A00826080937A0080917A0081602C
:101E500080937A0080917A00806880937A00109253
:101E6000BC021092BA021092B8028091D700816031
:101E70008093D70080EA8093D80089B5806189BDBE
:101E800089B5826089BD09B400FEFDCF0E947B0D3B
:101E90008091D8008F7C80618093D8008091E00091
:101EA000807F8093E0008091E1008E7E8093E1004E
:101EB0008DE08093E200559A209A8FEF9FEF9093E8
:101EC000CA028093C90280913C0390913D038830FF
:101ED0009105C8F49C012F5F3F4FF901EE0FFF1FE2
:101EE000E65EFC4F49E152E051834083880F991F21
:101EF000FC01E45DFC4F80E299E0918380833093A4
:101F00003D0320933C0380913C0390913D03883036
:101F10009105C8F49C012F5F3F4FF901EE0FFF1FA1
:101F2000E65EFC4F42E152E051834083880F991FE7
:101F3000FC01E45DFC4F8EE697E091838083309353
:101F40003D0320933C0380913C0390913D038830F6
:101F50009105C8F49C012F5F3F4FF901EE0FFF1F61
:101F6000E65EFC4F49E052E051834083880F991FA1
:101F7000FC01E45DFC4F80E297E091838083309325
:101F80003D0320933C0380913C0390913D038830B6
:101F90009105C8F49C012F5F3F4FF901EE0FFF1F21
:101FA000E65EFC4F42E052E051834083880F991F68
:101FB000FC01E45DFC4F82ED96E0918380833093D9
:101FC0003D0320933C0380913C0390913D03883076
:101FD0009105C8F49C012F5F3F4FF901EE0FFF1FE1
:101FE000E65EFC4F4DEF51E051834083880F991F0F
:101FF000FC01E45DFC4F89E798E091838083309396
:102000003D0320933C0380913C0390913D03883035
:102010009105C8F49C012F5F3F4FF901EE0FFF1FA0
:10202000E65EFC4F47EF51E051834083880F991FD4
:10203000FC01E45DFC4F8AE398E091838083309358
:102040003D0320933C0380913C0390913D038830F5
:102050009105C8F49C012F5F3F4FF901EE0FFF1F60
:10206000E65EFC4F4FEE51E051834083880F991F8D
:10207000FC01E45DFC4F8BEF97E09183808330930C
:102080003D0320933C0380913C0390913D038830B5
:102090009105C8F49C012F5F3F4FF901EE0FFF1F20
:1020A000E65EFC4F49EE51E051834083880F991F53
:1020B000FC01E45DFC4F8CEB97E0918380833093CF
:1020C0003D0320933C038CE792E00E94F10D8AE0EF
:1020D0008B8388E08C831E821D821F8289E291E0BF
:1020E0009A838983CE0101960E9452032A961FAEDD
:1020F0002A972B961FAE2B9780E22C968FAF2C97AA
:102100002E961FAE1EAE2E9760961FAE1EAE609727
:1021100062961FAE1EAE62978E01085F1F4F80E46D
:10212000E82EF12CCC24C3948DEB92E00E94FB01AD
:10213000892BD1F38DEB92E00E94FB01892BA1F357
:102140008D819E818034910518F01E821D82ECCF16
:102150008DEB92E00E940B03D82E8F81882329F00B
:102160006D2D8DEB92E00E94D5018B81D8122AC093
:10217000ED81FE81E00FF11F10821E821D826296AA
:102180001FAE1EAE62978885882371F22E961FAF10
:102190000EAF2E976096FFAEEEAE60972A96DFAC3C
:1021A0002A972C966FAD2C97062E000C770B2B964A
:1021B000BFAD2B97FE01319620E030E050E080E08B
:1021C00090E029C08C81D81216C08D819E81009725
:1021D00091F001979E838D838F81882309F4A4CF8A
:1021E00060E28DEB92E00E94D5016D2D8DEB92E0C7
:1021F0000E94D50199CF2FE12D1508F095CF8D8143
:102200009E819C012F5F3F4F3E832D83F801E80F95
:10221000F91FD08289CF4781411107C062963FAF35
:102220002EAF6297009731F417C02E3FAFEF3A07F9
:10223000D9F4F4CFE7E0F0E0EC0FFD1FE80FF91F51
:102240008081882349F062968EAD9FAD629701969A
:1022500062969FAF8EAF629762968EAD9FAD62978A
:10226000019609F461CF24C0D11005C0423219F49F
:1022700017825C250CC0511111C0A42EB12CA616DA
:10228000B70621F0BB2351F04D3341F4178200977C
:1022900029F04681442311F02F5F3F4F019631967C
:1022A0008034910509F0B7CF62963FAF2EAF6297A9
:1022B000BE01675B7F4F8AE193E00E948B06CE01EF
:1022C00001960E94520330CF1092C0021092BF02BA
:1022D00088EE93E0A0E0B0E08093C1029093C20248
:1022E000A093C302B093C40283E391E09093BE0233
:1022F0008093BD028FEF9FEF9093CA028093C90233
:1023000010920D0380914D03811113C01092480368
:10231000109247038DE192E090934A038093490322
:1023200086E390E090934C0380934B0381E080938D
:102330004D030E940905FC01A385B485109729F47B
:1023400087E493E0948783870BC08D919C911197CC
:10235000009711F0DC01F9CF87E493E08D939C9313
:102360002585368580914B0390914C03820F931FF6
:1023700096878587109211031092100385E491E0EF
:1023800090930F0380930E0380915B03811113C020
:10239000109256031092550383E592E090935803F0
:1023A000809357038FE290E090935A0380935903F0
:1023B00081E080935B030E940905FC01A385B4853D
:1023C000109729F485E593E0948783870BC08D915E
:1023D0009C911197009711F0DC01F9CF85E593E00E
:1023E0008D939C93258536858091590390915A034E
:1023F000820F931F9687858710923D0310923C03AE
:1024000080E1ECE1F3E0DF01982F1D929A95E9F766
:10241000ECE2F3E0DF011D928A95E9F781E591E0B6
:1024200090931B0380931A0308951F93FC0199272F
:102430008827BC01E89411911032E9F3193010F0AB
:102440001E30C8F31B3251F01D3249F4689406C0A7
:102450000E945A12610F711D811D911D119110531F
:102460001A30B0F33EF490958095709561957F4F4A
:102470008F4F9F4F1F910895FB01DC018D91813497
:102480001CF08B350CF4805E659161341CF06B356B
:102490000CF4605E861B611189F3990B0895BB27CC
:1024A0004A3031F4992322F4BDE2909581959F4FF3
:1024B0000C947012592F482F372F262F660F771F35
:1024C000881F991F660F771F881F991F620F731F40
:1024D000841F951F660F771F881F991F0895BB27BC
:1024E000FB015527AA27880F991FAA1FA41710F0D0
:1024F000A41B83955051B9F7A05DAA3308F0A95DDC
:10250000A193009779F7B111B1931192CB010C947B
:102510008912DC01FC01672F71917723E1F7329773
:1025200004C07C916D9370836291AE17BF07C8F3AE
:1025300008952F923F924F925F926F927F928F9267
:102540009F92AF92BF92CF92DF92EF92FF920F9342
:102550001F93CF93DF93CDB7DEB7CA1BDB0B0FB64C
:10256000F894DEBF0FBECDBF09942A883988488809
:102570005F846E847D848C849B84AA84B984C8849F
:10258000DF80EE80FD800C811B81AA81B981CE0F96
:10259000D11D0FB6F894DEBF0FBECDBFED0108957B
:1025A000EE0FFF1F0590F491E02D09940F931F93F8
:1025B000CF93DF938230910510F482E090E0E091B8
:1025C0006503F091660320E030E0A0E0B0E03097D2
:1025D00019F1408151810281138148175907C8F0D0
:1025E0008417950769F4109731F012960C9312979F
:1025F00013961C9327C0009365031093660322C0B3
:102600002115310519F04217530718F49A01BD013D
:10261000EF01DF01F801DBCF21153105F9F0281BAF
:10262000390B2430310580F48A819B816115710555
:1026300021F0FB019383828304C09093660380930F
:102640006503FE01329644C0FE01E20FF31F819341
:10265000919322503109398328833AC02091630332
:1026600030916403232B41F4209115013091160120
:10267000309364032093630320911301309114017C
:102680002115310541F42DB73EB740911701509106
:102690001801241B350BE0916303F0916403E217EA
:1026A000F307A0F42E1B3F0B2817390778F0AC0175
:1026B0004E5F5F4F2417350748F04E0F5F1F509352
:1026C0006403409363038193919302C0E0E0F0E0E0
:1026D000CF01DF91CF911F910F910895CF93DF9399
:1026E000009709F481C0FC01329713821282A091F5
:1026F0006503B0916603109781F420813181820FC8
:10270000931F20916303309164032817390751F513
:10271000F0936403E093630367C0ED0120E030E0D1
:10272000CE17DF0740F44A815B819E0141155105B8
:10273000F1F0EA01F5CFD383C28340815181840F48
:10274000951FC817D90759F488819981840F951F5F
:102750000296918380838A819B8193838283211552
:10276000310529F4F0936603E09365033DC0E90168
:10277000FB83EA8349915991C40FD51FEC17FD07DC
:1027800061F480819181840F951F0296E9019983FC
:102790008883828193819B838A83E0E0F0E01296B4
:1027A0008D919C911397009719F0FD01DC01F7CFF3
:1027B0008D919C9111979D012E5F3F4F820F931F2A
:1027C00020916303309164032817390769F4309727
:1027D00029F4109266031092650302C013821282DC
:1027E000B0936403A0936303DF91CF910895A0E0B9
:1027F000B0E0EDEFF3E10C949D12EC01009721F4B1
:10280000CB010E94D612B4C0FC01E60FF71F9C0159
:1028100022503109E217F30708F4A8C0D9010D913D
:102820001C91119706171707B0F00530110508F431
:102830009BC0C80104978617970708F495C00250FB
:102840001109061B170B019311936D937C93CF0114
:102850000E946E1389C05B01A01AB10A4C01800E60
:10286000911EA0916503B0916603612C712CE12C3F
:10287000F12C109709F446C08D919C911197A815E1
:10288000B905B1F56C0142E0C40ED11CCA14DB04D9
:1028900078F14C018A189B08640142E0C40ED11CF7
:1028A0001296BC9012971396AC91B5E0CB16D1045A
:1028B00040F0B282A38391828082D9016D937C9390
:1028C00009C00E5F1F4F800F911FF9019183808314
:1028D000EB2DFA2FE114F10431F0D7011396FC939C
:1028E000EE93129741C0F0936603E09365033CC0FA
:1028F0006816790608F43C017D0112960D90BC9192
:10290000A02DB7CF80916303909164038816990638
:10291000E1F466167706C8F48091130190911401D2
:10292000009741F48DB79EB740911701509118015F
:10293000841B950BE817F907C8F4F0936403E09340
:102940006303F901718360830FC0CB010E94D6122B
:102950007C01009759F0A801BE010E94C214CE016B
:102960000E946E13C70104C0CE0102C080E090E057
:10297000CDB7DEB7EEE00C94B91281E090E0F894A8
:102980000C94D214FB01DC0102C001900D92415065
:102990005040D8F70895FB01DC0101900D92002012
:0829A000E1F70895F894FFCF60
:1029A80000C18081000000FFFFFFFF00E100000080
:1029B800000000000067038000000000001502F519
:1029C80003B5033C02000000005203E502E20200E6
:1029D800000000D501D204F601EB01FB010B03E76F
:1029E800020000000038065F028C028B0200000023
:1029F800008B068F02DF02CE022903B902777269C3
:102A08007465200072656C6561736520007072657D
:102A180073732000636C69636B204D4F5553455F9A
:102A28004C45465400636C69636B204D4F555345C4
:102A38005F524947485400636C69636B204D4F559A
:102A480053455F4D4944444C4500636C69636B20B2
:102A58004D4F5553455F414C4C0072656C65617331
:102A680065204D4F5553455F4C4546540072656C83
:102A780065617365204D4F5553455F52494748542A
:102A88000072656C65617365204D4F5553455F4D08
:102A98004944444C450072656C65617365204D4F2F
:102AA8005553455F414C4C007072657373204D4F10
:102AB8005553455F4C454654007072657373204DFD
:102AC8004F5553455F5249474854007072657373B8
:102AD800204D4F5553455F4D4944444C4500707255
:102AE800657373204D4F5553455F414C4C006D6FD6
:102AF800766528002C200029005265636569766593
:102B080020536574004F6E6C7920416C61726D20A2
:102B1800697320616C6C6F7765642100537461720E
:0E2B2800742052656164696E67000D0A00003A
:00000001FF
